:10000000012AA000FF3A8417800529082A04031951
:10001000C928BB208413200880060E280000102861
:10002000A90A0319AA0F0D288006C92883169B0068
:1000300083161C141A089B0AC92883169A001C15DB
:1000400055309D00AA309D009C149C1825281C1139
:100050009B0AC9280F39AF000310AF0DAF0D1F0861
:10006000E0392F0401389F00643071209F149F18DD
:1000700037281E08B30083161E088312B200C92851
:100080000830AF002418AC2021088400220824196D
:10009000C120241DC3202008840023098417800563
:1000A00020088400AA0CA90C00082304031C2306C2
:1000B00080005D20AF0B5028C92821088400220849
:1000C0008006000080060800AC01AB00FF30AB07E3
:1000D000031CAC07031CC9280330AA00DF307220C0
:1000E0006628AA01E83EA900AA09FC30031C7B2867
:1000F000A90703187828A9070000AA0F782829184B
:100100008128A91C8528000085280800013EB00030
:100110000A30AB00AC019020B00B8B282D080800F2
:10012000AE01AD011030AF002A0DAD0DAE0D2B08A4
:10013000AD022C08031C2C0FAE020318A6282B08B6
:10014000AD072C0803182C0FAE070310A90DAA0D3C
:10015000AF0B942829080800AB01AC01B328AA0C06
:10016000A90CAB0DAC0DFF3E0318AF282C08AA005C
:100170002B08A900C928A909AA09A90A0319AA0ACA
:1001800008008004C628FF3A8005C728FF3A841774
:10019000800583138312031308003A08B8003E0653
:1001A000C400BD0803193729B90803193A293D08C5
:1001B000B9027F300318E028B907031C3929E32866
:1001C000B90703183C293C08B6003B08B700B8172C
:1001D000BE171830C300BC01BB01BA01F1280318D7
:1001E000FD28400836023F08031C3F0F37023E0837
:1001F000031C3E0F3802031C08294008B6023F08C2
:10020000031C3F0FB7023E08031C3E0FB802031445
:10021000BC0DBB0DBA0DB60DB70DB80DC30BEF2855
:10022000BA1B1A29B90803193929C40CB903C30A1E
:10023000C40DEF28421F362903182A294008B602A8
:100240003F08031C3F0FB7023E08031C3E0FB802D5
:10025000031C3629BC0F3629BB0F3629BA0F3629A5
:10026000BA0CBB0CBC0CB90A03193C294329C215B2
:100270003D294215B9013F29C214FF30B900BC0124
:10028000BB018030BA00C41B4629BA13C9283A08FA
:10029000C4007F303902C300031850290030A4295C
:1002A000BA17B901B6014308173CC3000318642903
:1002B0000830C307031CA2293A08B9003B08BA005A
:1002C0003C08BB00BC0171290830C302031C702923
:1002D0003C08B6003B08BC003A08BB00BA016429E0
:1002E000C307C30803197C290310B90CBA0CBB0C53
:1002F000BC0CB60CC30B74293918A229421F8729DC
:10030000B61F8729BC0F8729BB0F8729BA0A39086E
:10031000B6003C08B9003608BC003A08B6003B08F5
:10032000BA003608BB00C41FA029BC09BB09BA0922
:10033000B909B90FA029BA0FA029BB0A0319BC0A31
:100340003908C928C216FF30BC00BB00BA00B9008A
:10035000C928BB01BC019630C300C413BC1FBC2913
:10036000BC09BB09BA09B909B90FBB29BA0FBB2926
:10037000BB0A0319BC0AC417BC080319D729421FBA
:10038000CE29BC1FCE29BA0FCE29BB0FCE29BC0F58
:10039000CE290314BC0CBB0CBA0CC30A0830C3072B
:1003A0003A08B9003B08BA003C08BB00EC29BB087E
:1003B000031DEC290830C3023A08031DE829083060
:1003C000C3023908031DE7293C08C300F629B90117
:1003D000BB003908BA00B901BB1BF4290310B90DE1
:1003E000BA0DBB0DC303EC29C41FBB133908BC00F5
:1003F0004308B9003B08C3003A08BB004308BA00F1
:10040000C92883014030C20007309900831691014A
:10041000903083129F00303083169F00103091007F
:100420002F308500831285010130831687008312E7
:100430008701C801C70100301620C5001820C6007A
:1004400002301620CB001820CC00CE01CD01D00107
:10045000CF01D201D10104302A20C7003308C800DF
:100460000330480284300319470203183B2A043042
:10047000C7070318C80A033048022030031947028F
:100480000318462A0230C7070318C80A0230480278
:10049000BC30031947020318512A0230C70703185A
:1004A000C80A0230480258300319470203185C2A70
:1004B0000230C7070318C80A0130480290300319F8
:1004C00047020318672A0330C702031CC803013020
:1004D00048022C30031947020318722A0330C7025E
:1004E000031CC803C808031D7D2A0A3047020318ED
:1004F0007D2A0330C702031CC8034708B900480817
:10050000BA00A921F430C000FD30BF007430BE0035
:100510007F30BD00CD204721C7003A08C800CD0874
:10052000031D952ACE080319992ACD034D0A0319F4
:10053000CE034E084D04031DA62A4808CA004708EA
:10054000C900D201D101D001CF01BB2A83169B0182
:10055000831245081D2046081D20023083169B008B
:1005600083124B081D204C081D204608CA00450870
:10057000C900643064204A23051CC72AC83064209F
:10058000CF0A0319D00ACE010A30CD002323851CDF
:10059000D22AC8306420D10A0319D20ACE010A3007
:1005A000CD003623051DDC2AC8306420CB0A031990
:1005B000CC0ACE010A30CD00CC08031DE32A093055
:1005C0004B02031CE52ACC01CB0101304602031C7F
:1005D000F22A031DEF2A91304502031CF22AC601BC
:1005E0006430C50003104B0DB2004C0DB300B401D4
:1005F000B40DB50132084502A5004608A60033082F
:10060000031C330FA602A7013408031C340FA702F2
:10061000A8013508031C350FA802A81B212B2808A8
:10062000031D1F2B2708031D1F2B48082602031C30
:10063000212B031D1F2B47082502031C212B071606
:10064000222B07122B2AD008031D2A2B0B304F0216
:10065000031C322B0A30C5070318C60AD0010A3022
:10066000CF00352BC50A0319C60A0800D208031D9E
:100670003D2B0B305102031C452B0A30C502031CD5
:10068000C603D2010A30D100492BC503450A03191C
:10069000C60308004A08AA004908A90000308620BD
:1006A000D300CF230730A0000430A3000730A100FF
:1006B0000230A2000130A4000830A90040205408F4
:1006C000A9004020AA010130A900073084000830A9
:1006D0000120013064204A08AA004908A90001301D
:1006E0008620D300CF230730A0000430A3000730BA
:1006F000A1000230A2000130A4000430A900402073
:100700005408A9004020AA010130A9000730840044
:1007100008300120013064204A08AA004908A900D5
:1007200002308620D300CF230730A0000430A3007E
:100730000730A1000230A2000130A4000230A9005D
:1007400040205408A9004020AA010130A900073028
:10075000840008300120013064204C08AA004B08B6
:10076000A90000308620D300E7230730A000043022
:10077000A3000730A1000230A2000130A400103015
:10078000A90040205408A9004020AA010130A90076
:10079000073084000830012001306420080053082D
:1007A0000B3C031CE62BD623D400E62B03308A0037
:1007B00053088207C034F934A434B03499349234E5
:1007C0008234F83480349034BF34FF340800530846
:1007D000083C031CFB2BEE23D400FB2B03308A00C8
:1007E00053088207FF34FD34FC34DC349C349834E5
:0E07F00018341034003408006300FC2BFE2B7C
:02400E00A23FCF
:00000001FF
